:0A0000000C943B000C9495040C9442
:10000A0000000C9400000C9400000C9400000C9466
:10001A0000000C9400000C9400000C9400000C9456
:10002A0000000C9400000C9400000C9400000C9446
:10003A0040040C9400000C9400000C9400000C94F2
:10004A0000000C9400000C9400000C9471040C94B1
:10005A0000000C9400000C9400000C9400000000B6
:10006A00000000000600040068000000F894EE2773
:10007A00EFBBF1E0F5BFE5BFF8E1A895A4B7A77F0C
:10008A00A4BFF0936000E09360008DE0A2E0BB277C
:10009A00ED938A95E9F780E098E0A0E0B1E0ED936E
:1000AA000197E9F7EEE6F0E085919591009761F006
:1000BA00A591B59105901590BF01F00105900D929B
:1000CA000197E1F7FB01F0CFE0E0EEBBEFEFEDBF08
:1000DA00E8E0EEBFC0E0D3E00C94FF02E881E093D1
:1000EA007C0085E38A95F1F7E0917A00E064E09379
:1000FA007A000C94AB041A93E0917C00EF701E2FE7
:10010A00E0917800F0917900A981BA81ED93FC938E
:10011A00E12F18814FC0E0E0E0937C00ECE8E09327
:10012A007A000895A0910B03AF5FA0930B03E881B7
:10013A00AE1720F0E0E0E0930B03A8950C94AB0413
:10014A00E8E1E0936000E0E0E0936000E881E030FD
:10015A0039F0E8E1E0936000EFE0E0936000A895F1
:10016A000C94AB04E881E03011F0289801C0289A79
:10017A000C94AB040E94AD04E0EC0E94B104089513
:10018A000E94AD04E2E00E94B70458C10E94AD0487
:10019A00E881A1E00E941405E0680E94B1040C9471
:1001AA00AB040E94AD04E5E0EA930E94A504EA814B
:1001BA000E94B704239608951A930E94AD04E3E0BF
:1001CA00EA930E94A504E9810E94BE04EA93CADF69
:1001DA00E12F33C11A930E94AD04E0EA0E94BE04E3
:1001EA000E94B10441C11A93E981FA816B817C8131
:1001FA000E94620511F411E351C0E130A0E0FA0750
:10020A00A0E06A07A0E07A0711F417E247C0E230DB
:10021A00A0E0FA07A0E06A07A0E07A0711F418E163
:10022A003DC0E330A0E0FA07A0E06A07A0E07A0741
:10023A0011F413E133C0E430A0E0FA07A0E06A0742
:10024A00A0E07A0711F419E029C0E530A0E0FA0726
:10025A00A0E06A07A0E07A0711F417E01FC0E630B1
:10026A00A0E0FA07A0E06A07A0E07A0711F414E018
:10027A0015C0E730A0E0FA07A0E06A07A0E07A0715
:10028A0011F413E00BC0E830A0E0FA07A0E06A0717
:10029A00A0E07A0711F411E001C010E0EAE2EA9363
:1002AA001A936EDFE9E2EA93E8EAEA9369DFE8E2A1
:1002BA00EA93E3E0EA9364DF1881259608951A9396
:1002CA000E94AD04E2E0EA930E94A504EB85A0E156
:1002DA00EA02F001E05DEA930E94A504EC81EA9348
:1002EA000E94A504AF81B88589859A85E3E00E94BA
:1002FA003105EA930E94A504EF81E295E07FEE0FB3
:10030A00EA930E94A5040E94C6040E94C604EA81D8
:10031A00E295E07FEE0FEE0FA981EA2BEA930E94A5
:10032A00A50410E0E9811E1760F40E94C904AD819A
:10033A00BE81AE0FBF1FEC91EA930E94A5041F5F16
:10034A00F1CFE0E0EA930EDF18812C9608951A9314
:10035A000E94AD04E3E0EA930E94A504E981A0E1CA
:10036A00EA02F001E05AEA930E94A50410E01E3066
:10037A0090F40E94CC04ED5EFC4FDF010E94C90498
:10038A00EA0FFB1FFF93EF930E94C604AF91BF9140
:10039A00EC931F5FECCFE0E0EA93E4DE89800E94F1
:1003AA00CC04EC5EFC4F0E94D104E3E00E942505D8
:1003BA00E87FF770607070700E94D804EB5EFC4FA3
:1003CA000E94D104E5E00E943105E770F070607088
:1003DA007070A0910C03B0910D0380910E0390915F
:1003EA000F030E940F050E94D804E85EFC4FE081CB
:1003FA00EF70AE2E0E94CC04E85EFC4FE081E07400
:10040A0011F0E1E001C0E0E0DE2E10E01A15A0F4E0
:10041A000E94C904CF01E05FFC4FBF010E94CC04D7
:10042A00ED5EFC4FDF01FC013696AE0FBF1FEC916B
:10043A00DB01EC931F5FEACFE1E018812296089571
:10044A00E0E6EA93E4E0EA93EA81EE0FEE0FEA933C
:10045A00A8DE7CC21A93EEE0EA93AEDEF0E0F595F0
:10046A00E7950E9446051E2FE12F19910895F2DFA4
:10047A00AE2FE881EA1759F0EFE0EA93E0EEEA934B
:10048A00EA81E295E07FEE0FEA938BDEF0CF5EC25F
:10049A00289A209A08956EDEEFE0EA93E8E0EA935C
:1004AA006FDEE4E0EA93E3DFE88186D29CDEE0E6F1
:1004BA0089D2E0E787D2E1E0EA93C2DFEBE2EA938E
:1004CA00E3EAEA935DDEE0E0EA93D1DF3FC2E88146
:1004DA00EA933DDFE0910C03F0910D0360910E0366
:1004EA0070910F03A72DBB27882799270E946605BD
:1004FA0019F4E3E0EA1509F03DC0E0911003F0E0D9
:10050A00F0700E944105E0930403F0930503A09163
:10051A001103B0E0E6E00E941C05E370F070A091C0
:10052A000403B0910503EA2BFB2BE0930403F09339
:10053A000503E0911103F0E0EF73F0700E943D05AE
:10054A00E0930603F0930703A0910603B091070313
:10055A00E0911203F0E00E944605EF70F070EA2B7A
:10056A00FB2BE0930603F0930703E0911203E37079
:10057A009E2EF29AEBC1E881E17019F0E0E0EA936D
:10058A00A6DFE881E27019F0E1E0EA93A0DFDEC1BC
:10059A00EFE0EA93E0E1EA93E0E0EA9302DE08950D
:1005AA000E946B05ECE2EA9307DE1E2FEDE2EA9366
:1005BA0003DE0E2F0FDE3E2FECE2EA93E0E0EA9331
:1005CA00DFDDEDE2EA93E0E0EA93DADD17FD02C04F
:1005DA0015FF01C00AC0E02FE87321F0E4E0EA93B6
:1005EA005ADF02C03A93C7DF01C0D2DF0E9470050A
:1005FA00249608959FD039D14BDF05D17894E1E054
:10060A00EA939EDDE7D087DDF1D0E4E0EA9343DFA9
:10061A00E6B1F0E0F595E795E095EF705E2E309B38
:10062A0005C0E52DE05F4E2E752C04C0452CE52D46
:10063A00E05F7E2EF39B12C0F3984C9B03C0E1E06F
:10064A006E2A02C0EEEF6E224D9B03C0E2E06E2AD4
:10065A0002C0EDEF6E22E6E0EA9340DDF09B42C075
:10066A00F098E0910003F09101030E945305E09392
:10067A000803E0910003E370E295E07FEE0FEE0FCE
:10068A00E0930903E9E0F3E00F01A081E09102039E
:10069A00F09103030E944F05EF73EA2BD001EC930C
:1006AA00E0910203EF70E295E07FE0930A03EAE04B
:1006BA00F3E00F01A081E62DE370EA2BD001EC9361
:1006CA00E0E0EA93E42D78D1E8E0F3E0FA93EA93E4
:1006DA00E0E0EA93EA93EA93E3E0EA93F0DDE0E00C
:1006EA00EA9354DDF29B1FC0F29890FE02C05E9A14
:1006FA0001C05E9891FE02C05F9A01C05F98E091C6
:10070A000503F070E370E0938900E0910403E0933D
:10071A008800E0910703F070E370E0938B00E091AA
:10072A000603E0938A00F19B02C05B9A01C05B98C2
:10073A006FCFFFCFE0E0E5B9E4B9E8B9E7B9EBB9C3
:10074A00EAB9E4BDE5BDE6BDE7BDE8BDE0938000DA
:10075A00E0938100E0938500E0938400E0938700B2
:10076A00E093860035D1E0E0E093B600E093B00074
:10077A00E093B100E093B200E093B300E093B400D9
:10078A00E0936900EDBBECBBE0936800E2E0E09324
:10079A006E00E0E0E0936F00E0937000E093C00029
:1007AA00E093C100E093C200E093C500E093C40067
:1007BA00E0E8E0BFE0E0E0937B00E0937F00E093B5
:1007CA007A00E0937C00E0937E00ECBDEDBDE093FF
:1007DA00BC000895259A239AEDB5E160EDBDECB50C
:1007EA00E061ECBDECB5E064ECBD0895E091690010
:1007FA00E260E0936900E0916900EE7FE0936900AE
:10080A00E89AE09A0895E4B5EE7FE4BDE4B5E260C3
:10081A00E4BDE4B5E77FE4BDE5B5EB7FE5BDE5B54D
:10082A00E260E5BDE5B5E160E5BDE9EFE7BDE09170
:10083A008000E068D7D0EF7BD5D0E062D3D0EF7EDE
:10084A00D1D0E160CFD0E260E0938000E0918100F6
:10085A00E860CDD0EF7ECBD0E160C9D0ED7FC7D0C4
:10086A00EB7FE0938100B4D00895569A579A539A31
:10087A00219A229A0895C0D0E4E6EA9353DCAFE2C3
:10088A00B3E0ED91FD913196FE93EE93E436A0E04C
:10089A00FA0729F4E0E0E0932F03E0933003E091B4
:1008AA002F03F0913003309719F4F09AF19A08C0A7
:1008BA00A0912F03B09130031F9711F4F09AF19889
:1008CA00A0913103AF5FA0933103A53021F4E0E09A
:1008DA00E0933103F39A26C08FD00E946B0500E0A3
:1008EA0010E0EDB7FEB73197FA93EA931F930F938F
:1008FA0002DC0F911F913E2F363041F40093000322
:10090A0010930103E7E0EA93E9DB06C0373021F4EC
:10091A00E2E0F3E0008311830E947005249602C08E
:10092A006BD03EDEE991EFBFF991E991B991A991B6
:10093A009991899179916991F990199009901895ED
:10094A00E881EEBDEDB5E7FFFDCFEEB5219608953E
:10095A00E1E0EA930C94B700EA93F2DFE0E0EA936D
:10096A000C94B700EA93ECDFE981EA93E9DFE881C6
:10097A00F3CFEA93E5DFE0E0EA93E2DF1E2FE0E05F
:10098A000895E0E0EA93DCCFE12FF0E00895E981F1
:10099A00AEE0EA9FF0010895E081F0E00E94580578
:1009AA00DF01CB010895E0930C03F0930D036093EC
:1009BA000E0370930F03EBCFF0E00E9458050E94DC
:1009CA005D050895EA93E0E6EA93EA930C94D6006B
:1009DA00E0E0E0938900E0938800E0938B00E093E5
:1009EA008A000895E0938000E09180000895E093E2
:1009FA008100E091810008950A921A92FA926A930C
:100A0A007A938A939A93AA93BA93EA93FA93EFB74B
:100A1A00EA930895EA2BFB2B682B792B0895EE2392
:100A2A000E2EEA2F19F0EE0F0A94E9F70895EE2335
:100A3A000E2EFD0121F0F595E7950A94E1F7089548
:100A4A00EE230E2EFD01BC0131F0EE0FFF1F661FD3
:100A5A00771F0A94D1F70895EE230E2EFD01BC01EB
:100A6A0031F076956795F795E7950A94D1F7089549
:100A7A00EE0FFF1FEE0FFF1FEE0FFF1FEE0FFF1F00
:100A8A000895F595E795F595E795F595E795F59523
:100A9A00E7950895F695E795F695E795F695E7951E
:100AAA00F695E79508956F2F660F660B762F0895D2
:100ABA007A936A93FA93EA93089530976040704064
:100ACA000895EA17FB076807790708953A932A9366
:100ADA001A930A9308953B812A81198108810895FE
:00000001FF
